:020000040000FA
:0400000071303A28F9
:08000800A000030EA100831209
:1000100005191028831601178312B23081002B288E
:1000200083160113831203140B190310A80DA90DD5
:10003000AA0DAB0DAC0DAC16FF302C02031D2B2806
:10004000FA302B02031D2B2831152A08AF0029088E
:10005000AE002808AD008B100B11210E8300A00EFE
:04006000200E090065
:0C007400203084008001840A80300402E7
:10008000031C3C281230B000722183160C30850509
:1000900087018312850187010730990000309A009B
:1000A000103083168E008312603083168F00831207
:1000B0000030831691009F008312C83083168100A0
:1000C000831231309000003083168C008312103080
:1000D0008B00831600309B001C141A088312BC008E
:1000E000831610309B001C141A088312BD0083165F
:1000F0002F309B001C141A088312C3008B21831617
:1001000020309B001C141A088312C2000130C20860
:100110000319C20081018E018F010B118B100B108E
:100120008C018B17A2203119A5205421B30BA028D4
:10013000031085190314B90DF03039020319FD209D
:100140008E21922864003210080031110130B7006E
:100150008B132030370783169B001C141A08831258
:10016000A4001030370783169B001C141A08831252
:10017000A300A6000230A6060030370783169B00B6
:100180001C141A088312A200A7000130A7068B17BF
:10019000321CD02822090339A200A309A409A50909
:1001A00024082F02031DF72823082E02031DE5282B
:1001B00022082D02031DF72801303702031DE52810
:1001C0003D18E5283D143E14852126082E02031D06
:1001D000F72827082D02031DF72801303702031DD9
:1001E000F6283D1CF6283D103E148921F728B70A51
:1001F0000230370203180800A8280130B600B30007
:10020000B400B500B70085018701B113A220B30B7C
:100210002329031085190314B90DF030390203198D
:100220004A29B41F8501B41F8701B40B232937085D
:10023000B6080319B60003192129FF30850087008D
:10024000B6039630B400311D06293111321C2D2918
:100250002D090339AD00AE09AF092F1C06298E0107
:100260008F010C1C06290C102E1E06298B13203022
:100270003707BB002F08BA005D2110303707BB00DD
:100280002E08BA005D2100303707BB002D08BA00E8
:100290005D218B1785018701B70AB601023037024D
:1002A000031C06298B2108003E1C08003E1010305C
:1002B000BB003D08BA005D2108008B133A08831685
:1002C0001C159A0083123B0883169B0055309D0035
:1002D000AA309D009C1464009C186B291C11831289
:1002E0008B170800FF30D4000230D5000C30D60048
:1002F000BA30D7003730D800DA30D9006F30DA00A2
:10030000B830DB000230C10008000130BD00DD1450
:100310000800DD1008003D18DD1408005C18051603
:10032000DC1885165C190514DC1985145C1A871411
:10033000DC1A07155C1B0714DC1B87165D180716F3
:10034000DD1887155C1C0512DC1C85125C1D051070
:10035000DC1D85105C1E8710DC1E07115C1F07105A
:10036000DC1F87125D1C0712DD1C87118F08031923
:1003700008008F01C10B08004208C1005408DE00CC
:100380000723D4005508DE000723D5005608DE00F9
:10039000541C0723D6005708DE00D41C0723D700BF
:1003A0005808DE00541D0723D8005908DE00D41D6C
:1003B0000723D9005A08DE00541E0723DA005B0821
:1003C000DE00D41E0723DB005C08C6005D08C70002
:1003D000CA0B002A5408CA008B13831640309B00B6
:1003E0001C141A0883125405031D5C148316503024
:1003F0009B001C141A0883125405031D5C108B17F4
:10040000CB0B182A5508CB008B13831641309B0069
:100410001C141A0883125505031DDC148316513071
:100420009B001C141A0883125505031DDC108B1742
:10043000CC0B302A5608CC008B13831642309B001D
:100440001C141A0883125605031D5C1583165230BE
:100450009B001C141A0883125605031D5C118B1790
:10046000CD0B482A5708CD008B13831643309B00D1
:100470001C141A0883125705031DDC15831653300C
:100480009B001C141A0883125705031DDC118B17DF
:10049000CE0B602A5808CE008B13831644309B0085
:1004A0001C141A0883125805031D5C168316543059
:1004B0009B001C141A0883125805031D5C128B172D
:1004C000CF0B782A5908CF008B13831645309B0039
:1004D0001C141A0883125905031DDC1683165530A7
:1004E0009B001C141A0883125905031DDC128B177C
:1004F000D00B902A5A08D0008B13831646309B00ED
:100500001C141A0883125A05031D5C1783165630F3
:100510009B001C141A0883125A05031D5C138B17C9
:10052000D10BA82A5B08D1008B13831647309B00A0
:100530001C141A0883125B05031DDC178316573041
:100540009B001C141A0883125B05031DDC138B1718
:10055000D20BC02A5608D2008B13831648309B005A
:100560001C141A0883125505031D5D148316583098
:100570009B001C141A0883125705031D5D108B176E
:10058000C4015C18C40ADC18C40A5C19C40ADC196A
:10059000C40A5C1AC40ADC1AC40A5C1BC40ADC1B49
:1005A000C40A5D18C40AC5014618C50AC618C50A9A
:1005B0004619C50AC619C50A461AC50AC61AC50A81
:1005C000461BC50AC61BC50A4718C50A3D1CFE2A9C
:1005D000430845020318F52A450844020318080099
:1005E0004608DC004708DD00080043084402031801
:1005F00008004608DC004708DD0008004408450202
:10060000031808004608DC004708DD000800C001A8
:10061000DE080319DE035E184014DE1A4014400899
:10062000C0015E1C4014DE1E4014C005C00C5E0CF0
:020630000800C0
:084000000E000300040008009B
:02400E00CC33B1
:10420000010078007A007C007E007B0079007F004E
:104210007D007A0078007E007C00FF00FF00FF0038
:104220000000F200F600FA00FE00F200F600FA00CC
:10423000FE00F200F600FA00FE00FF00FF00FF00A3
:10424000100005000500050005000900090009002F
:1042500009000D000D000D000D00FF00FF0005001E
:10426000FF00FF00FF00FF00FF00FF00FF00FF0056
:10427000FF00FF00FF00FF00FF00FF00FF00FF0046
:104280000800800002000800040010000400200064
:1042900004000200FF00FF00FF00FF00FF00FF001E
:1042A00001000100010004000800040010000400E7
:1042B00080000400FF00FF00FF00FF00FF00FF0080
:1042C000FF00FF00FF00FF00FF00FF00FF00FF00F6
:1042D000FF00FF00FF00FF00FF00FF00FF00FF00E6
:1042E000FF00FF00FF00FF00FF00FF00FF00FF00D6
:1042F000FF00FF00FF00FF00FF00FF00FF00DD00E8
:00000001FF
